:100000000C9465020C94A9020C94A9020C94A90208
:100010000C94A9020C94A9020C94A9020C94A902B4
:100020000C94A9020C94A9020C94430D0C94150E87
:100030000C942B1C0C94A9020C94A9020C94A902F8
:100040000C94A9020C94A9020C94A9020C94A90284
:100050000C94A9020C94981C0C94A9020C94A9026B
:100060000C94A9020C94A9020C94A9020C94A90264
:100070000C94A9020C94A9020C94A9020C94A90254
:100080000C94A9020C94A9020C94A9020C94A90244
:100090000C94A9020C94A9020C94A9020C94A90234
:1000A0000C94A9020C94A9020C94A90235001E001C
:1000B0001F0020002100220023002400250026002C
:1000C00027002A002B0014001A0008001500170052
:1000D0001C0018000C00120013002A002900040064
:1000E0001600070009000A000B000D000E000F00AB
:1000F00033003400E1001D001B000600190005005C
:100100001100100036003700380028000030E000F1
:10011000E200E30003522C002C0004525000510076
:1001200052004F0035001E001F0020002100220059
:10013000230024002500260027002A002B0014009D
:100140001A00090013000A000D000F0018001C001F
:1001500033002A00290004001500160017000700CC
:100160000B00110008000C0012003400E1001D001B
:100170001B000600190005000E00100036003700B5
:10018000380028000030E000E200E30003522C00B9
:100190002C0004525000510052004F0035001E0048
:1001A0001F0020002100220023002400250026003B
:1001B00027002A002B0034003600370013001C00F3
:1001C00009000A00060015000F002A00290004009B
:1001D0001200080018000C0007000B0017001100A7
:1001E00016003800E100330014000D000E001B0063
:1001F000050010001A0019001D0028000030E00062
:10020000E200E30003522C002C0004525000510085
:1002100052004F0035001E001F0020002100220068
:10022000230024002500260027002A0035021E0294
:100230001F0220022102220223022402250226029A
:1002400027022A0001003A003B003C003D003E002E
:100250003F002D022E022F02300231020100400029
:100260004100420043004400450000530153025343
:100270000050010001000100010001000100010027
:1002800001000100AB00AA00A900AE0035001E006D
:100290001F0020002100220023002400250026004A
:1002A00027002A0035001E001F0020002100220028
:1002B000230024002500260027002A0001003A0020
:1002C0003B003C003D003E003F002D002E002F0073
:1002D0003000310001004000410042004300440072
:1002E000450000530153025300500100010001007A
:1002F000010001000100010001000100AB00AA00A3
:10030000A900AE002A0354006800650020005000D8
:10031000720065006F006E006900630020004B00F2
:100320006500790062006F006100720064000000E7
:100330002C034F007200740068006F006C006900AD
:100340006E0065006100720020004B0065007900BE
:1003500062006F006100720064007300000004031B
:10036000090409027400040100A0FA090400000154
:1003700003010100092111010001223F000705814D
:100380000308000A09040100010301020009211108
:10039000010001224D000705820308000A0904023A
:1003A00000010300000009211101000122360007AD
:1003B00005830308000A0904030002030000000982
:1003C00021110100012220000705840320000107FC
:1003D0000504032000011201100100000008EDFED9
:1003E00061600100010200010631FF0974A10109E9
:1003F00075150025FF9520750881020976150025E1
:10040000FF952075089102C005010980A1018502B0
:1004100016010026B7001A01002AB70075109501D1
:100420008100C0050C0901A1018503160100269C6D
:10043000021A01002A9C02751095018100C0050175
:100440000902A1010901A1000509190129051500E9
:10045000250195057501810295017503810105014D
:10046000093009311581257F950275088106093803
:100470001581257F950175088106050C0A3802153E
:1004800081257F950175088106C0C005010906A177
:1004900001050719E029E715002501950875018177
:1004A0000295017508810105081901290595057551
:1004B0000191029501750391010507190029FF15A6
:1004C0000025FF950675088100C011241FBECFEFDF
:1004D000DAE0DEBFCDBF04B603FE24C08091F10197
:1004E0009091F201A091F301B091F4018730904B0B
:1004F000A740B04BB9F41092F1011092F2011092A2
:10050000F3011092F40114BE84B7877F84BF88E1A1
:100510000FB6F89480936000109260000FBEE0E088
:10052000F8E3099511E0A0E0B1E0E0EEF9E402C0E3
:1005300005900D92A435B107D9F711E0A4E5B1E01B
:1005400001C01D92A13FB107E1F70E94720A0C940D
:10055000EE240C94000061110DC0FC0182818823FF
:1005600031F085EE0E9426110E94272303C085EEFC
:100570000E94EE1180E090E00895089508950E9491
:10058000D1026E9A769A8DEB92E0892B11F00C9441
:10059000BD0208958EEB92E0892B11F00C94BE02FF
:1005A0000895279A2F988FEF9FEF9093870080935D
:1005B00086008AE08093800089E1809381000C941A
:1005C000D02281110BC080918000877F80938000B2
:1005D00010928D0010928C002F9808952F988330E0
:1005E00041F4809180008860809380008FEF9FEFBE
:1005F00012C09091800098609093800023E030E0DA
:10060000281B3109220F331F8FEF9FEF02C09695F1
:1006100087952A95E2F790938D0080938C0008953A
:100620008B3B910568F4883A910530F5853A910540
:10063000C0F48430910598F4019709F06FC071C03F
:10064000803E910508F46AC0883E910540F09C0107
:10065000205F31092031310508F060C05CC09C0189
:10066000A1C0853A910509F45FC0863A910509F465
:100670005EC023E830E496C0883A910509F45AC078
:10068000893A910509F459C08A3A910509F458C08C
:100690008B3A910509F457C08C3A910509F456C07C
:1006A0008D3A910509F455C0803B910509F454C079
:1006B0008E3A910509F453C08F3A910509F452C05E
:1006C000813B910509F451C0823B910509F450C06A
:1006D000833B910509F44FC0843B910509F44EC05A
:1006E000853B910509F44DC0863B910509F44CC04A
:1006F000873B910509F44BC0883B910509F44AC03A
:10070000893B910509F449C08A3B910509F048C02D
:100710002AE236E447C09C01306544C020E030E066
:1007200041C021E030E03EC021E830E43BC022E897
:1007300030E438C022EE34E435C029EE34E432C06F
:100740002AEE34E42FC025EB34E42CC026EB34E44D
:1007500029C027EB34E426C02CEC34E423C02DEC74
:1007600034E420C023E835E41DC02AE835E41AC08B
:1007700022E935E417C024E935E414C021E236E467
:1007800011C023E236E40EC024E236E40BC025E2B9
:1007900036E408C026E236E405C027E236E402C0AB
:1007A00020E034E4C901089508959CE0799FF001A8
:1007B00011249CE3899FE00DF11D1124E60FF11D2A
:1007C000EE0FFF1FE455FF4F25913491C9010895A5
:1007D000880F991F845D9040FC0125913491C901D7
:1007E0000895880F991F84559F4FFC0125913491DE
:1007F000C90108950E94D5039C019A9581159F41D6
:1008000010F4C9010895C90190528115904128F44E
:10081000C9019F700E94F1030895C9019053811589
:10082000904120F4C9019927906C0895C901905412
:10083000409728F4C9018F709927946D089520314D
:1008400080E4380719F480E091ED0895213190E4B7
:10085000390719F480E090ED0895223140E434071F
:1008600019F480E092ED0895233180E4380719F4FB
:1008700080E093ED0895211590E5390769F40E9411
:1008800015162FEF44E38CE0215040408040E1F703
:1008900000C000000C94BD1C213090E5390731F4F4
:1008A0008091D00181608093D0010895C901905555
:1008B0008115904108F062C0432F55274F7055278E
:1008C00041305105F9F4C90174E0880F991F7A95F8
:1008D000E1F788279370B901E3E0660F771FEA9587
:1008E000E1F760767727862B972B9C682370332758
:1008F00002C0440F551F2A95E2F74F715527842BEC
:10090000952B08954230510529F4922F8827816F45
:10091000906A089543305105B9F4C90153E0880F36
:10092000991F5A95E1F7807E97702370332741E035
:1009300050E002C0440F551F2A95E2F74F7155272A
:10094000842B952B9C6808954430510549F5C901C5
:1009500043E0880F991F4A95E1F7807E97702370D6
:10096000332741E050E002C0440F551F2A95E2F7BB
:100970004F715527842B952B9A680895C90190577C
:100980008115904120F4C9019F7090620895C901BA
:1009900090588115904120F4C9019F70906A089584
:1009A000203E3105E0F4203C310568F52133310566
:1009B00009F475C048F42932310509F46BC02A32B4
:1009C000310509F07BC075C02933310501F12238AA
:1009D0003105E9F02533310509F070C051C0233EDF
:1009E0003105B1F140F4203E3105D1F0223E310510
:1009F00009F064C01CC0263E310579F1273E31055F
:100A000009F05CC038C0C9010E94E80308958091D4
:100A1000E10180FD02C081FF51C080EE90E04FC037
:100A20008091E10180FFF9CF89E390E048C0809197
:100A3000E10182FF0AC08091E10184FF03C080E0F0
:100A400090E03DC083EE90E03AC082EE90E037C087
:100A50008091E10182FFEFCFF8CF8091E10183FF28
:100A600007C08091E10184FDEACF87EE90E027C0C6
:100A700086EE90E024C08091E10183FFF2CFF8CFB1
:100A80008091E10185FF03C089E290E018C085E311
:100A900090E015C08091E10185FDF9CFF5CF8091FF
:100AA000E10186FF03C08AE290E009C081E390E0A3
:100AB00006C08091E10186FDF9CFF5CFC9010E9402
:100AC0001003089508955F926F927F928F929F9284
:100AD000AF92BF92CF92DF92EF92FF920F931F934C
:100AE000CF93DF93CDB7DEB72A970FB6F894DEBF6A
:100AF0000FBECDBF9E012F5F3F4F4E018BE0880E92
:100B0000911C60E070E000E010E0E12CF12CC12CC1
:100B1000D12CA12CB12C8AE0782E622E532E41E0EC
:100B200050E0E4E1F1E0A62DB52D872D01900D9266
:100B30008A95E1F7F901819191919F01FC01E07F94
:100B4000FF27E032F10559F48F709927FA0102C0AE
:100B5000EE0FFF1F8A95E2F7AE2ABF2A37C0E033B7
:100B6000F10559F48F709927FA0102C0EE0FFF1FAB
:100B70008A95E2F7CE2ADF2A29C0E034F10559F43C
:100B80008F709927FA0102C0EE0FFF1F8A95E2F7D6
:100B9000EE2AFF2A1BC0E035F10559F48F70992722
:100BA000FA0102C0EE0FFF1F8A95E2F70E2B1F2BF2
:100BB0000DC0E036F10551F48F709927FA0102C09B
:100BC000EE0FFF1F8A95E2F76E2B7F2B2815390554
:100BD00009F0A7CF94B18A2D8095892384B985B176
:100BE0008A2985B997B18C2D8095892387B988B1D9
:100BF0008C2988B99AB18E2D809589238AB98BB1B9
:100C00008E298BB99DB1802F809589238DB98EB1A6
:100C1000802B8EB990B3862F8095892380BB81B3BA
:100C2000862B81BB2A960FB6F894DEBF0FBECDBFD0
:100C3000DF91CF911F910F91FF90EF90DF90CF90B8
:100C4000BF90AF909F908F907F906F905F9008952E
:100C50005F926F927F928F929F92AF92BF92CF924C
:100C6000DF92EF92FF920F931F93CF93DF93CDB755
:100C7000DEB768970FB6F894DEBF0FBECDBF85B75D
:100C8000806885BF85B7806885BF0E9463059E0127
:100C90002F5F3F4F4E0189E1880E911C60E070E0AC
:100CA00000E010E0E12CF12CC12CD12CA12CB12CB6
:100CB00098E1792E622E532E41E050E0EEE1F1E012
:100CC000A62DB52D872D01900D928A95E1F7F9019A
:100CD000819191919F01FC01E07FFF27E032F105B6
:100CE00059F48F709927FA0102C0EE0FFF1F8A9501
:100CF000E2F7AE2ABF2A37C0E033F10559F48F700E
:100D00009927FA0102C0EE0FFF1F8A95E2F7CE2A5B
:100D1000DF2A29C0E034F10559F48F709927FA01D0
:100D200002C0EE0FFF1F8A95E2F7EE2AFF2A1BC0D2
:100D3000E035F10559F48F709927FA0102C0EE0FE2
:100D4000FF1F8A95E2F70E2B1F2B0DC0E036F10531
:100D500051F48F709927FA0102C0EE0FFF1F8A9598
:100D6000E2F76E2B7F2B2815390509F0A7CF94B138
:100D70008A2D8095892384B985B18A2985B997B14F
:100D80008C2D8095892387B988B18C2988B99AB12F
:100D90008E2D809589238AB98BB18E298BB99DB10F
:100DA000802F809589238DB98EB1802B8EB990B319
:100DB000862F8095892380BB81B3862B81BB1092BF
:100DC00055011092540110925F0110925E01109231
:100DD0005701109256011092610110926001109219
:100DE0005901109258011092630110926201109201
:100DF0005B0110925A0110926501109264011092E9
:100E00005D0110925C0110926701109266018FEBF8
:100E100092E0892BB9F068960FB6F894DEBF0FBE4A
:100E2000CDBFDF91CF911F910F91FF90EF90DF9099
:100E3000CF90BF90AF909F908F907F906F905F907A
:100E40000C94BF0268960FB6F894DEBF0FBECDBFFC
:100E5000DF91CF911F910F91FF90EF90DF90CF9096
:100E6000BF90AF909F908F907F906F905F9008950C
:100E70005F926F927F928F929F92AF92BF92CF922A
:100E8000DF92EF92FF920F931F93CF93DF93CDB733
:100E9000DEB7A2970FB6F894DEBF0FBECDBF7E01BE
:100EA00049E1E40EF11C2EE5C22E21E0D22E5E01B6
:100EB00053E2A50EB11C3AE0532E470101E010E0C9
:100EC00048E1642E55E0752EE4E1F1E0D401852D72
:100ED00001900D928A95E1F7F701819191917F013F
:100EE0009C01207F33272032310589F424B18F7093
:100EF0009927A80102C0440F551F8A95E2F7CA013D
:100F0000242B24B995B18095892385B94FC020330E
:100F1000310589F427B18F709927F80102C0EE0FCF
:100F2000FF1F8A95E2F7CF012E2B27B998B1809544
:100F3000892388B93BC02034310589F42AB18F70E8
:100F40009927A80102C0440F551F8A95E2F7CA01EC
:100F5000242B2AB99BB1809589238BB927C02035D2
:100F6000310589F42DB18F709927F80102C0EE0F79
:100F7000FF1F8A95E2F7CF012E2B2DB99EB18095E8
:100F800089238EB913C02036310581F420B38F70C8
:100F90009927A80102C0440F551F8A95E2F7CA019C
:100FA000242B20BB91B38095892381BB50EA5A95AD
:100FB000F1F7BE016F5F7F4F80E090E020E030E00E
:100FC000EEE1F1E0DE011196462D01900D924A9579
:100FD000E1F7FB0141915191BF01FA01E07FFF2749
:100FE000E032F10511F4E3B113C0E033F10511F47F
:100FF000E6B10EC0E034F10511F4E9B109C0E03505
:10100000F10511F4ECB104C0E036F105B9F4EFB12B
:10101000F0E04F70552702C0F595E7954A95E2F745
:10102000E0FD08C0A801022E02C0440F551F0A941B
:10103000E2F702C040E050E0842B952B2F5F3F4F3A
:101040002C30310509F0BCCFF60120813181281701
:10105000390721F091838083709200010E9463051B
:10106000F2E0CF0ED11CEA14FB0409F02DCF8091E1
:1010700000018823A1F1815080930001882339F079
:101080008FE99FE00197F1F700C0000028C0809130
:101090005E0190915F01909355018093540180917E
:1010A0006001909161019093570180935601809166
:1010B000620190916301909359018093580180914E
:1010C00064019091650190935B0180935A01809136
:1010D00066019091670190935D0180935C018AECB9
:1010E00092E0892B11F00E94CA0281E0A2960FB60D
:1010F000F894DEBF0FBECDBFDF91CF911F910F914E
:10110000FF90EF90DF90CF90BF90AF909F908F9027
:101110007F906F905F900895E82FF0E0EE0FFF1F33
:10112000EC5AFE4F8081918108950895809171015C
:101130000895CF93DF9300D01F92CDB7DEB72091F3
:10114000E701243021F523E029839B838A832093C0
:10115000E9008FEF06C095ED9A95F1F7000088231E
:1011600029F09091E800815095FFF5CF8091E8003B
:1011700085FF0DC040E050E063E070E0CE010196D5
:101180000E94280B8091E8008E778093E8000F90F2
:101190000F900F90DF91CF910895CF93DF9300D000
:1011A0001F92CDB7DEB72091E701243029F522E068
:1011B00029839B838A8383E08093E9008FEF06C0B5
:1011C00095ED9A95F1F70000882329F09091E800B9
:1011D000815095FFF5CF8091E80085FF0DC040E07C
:1011E00050E063E070E0CE0101960E94280B8091F0
:1011F000E8008E778093E8000F900F900F90DF91BA
:10120000CF9108952091E7012430F9F422E0209352
:10121000E9002FEF06C035ED3A95F1F700002223E3
:1012200029F03091E800215035FFF5CF2091E800FA
:1012300025FF0BC040E050E065E070E00E94280B05
:101240008091E8008E778093E8000895CF93DF9334
:10125000EC018091E701843041F581E08093E90061
:101260008FEF06C095ED9A95F1F70000882329F0DD
:101270009091E800815095FFF5CF8091E80085FFBF
:1012800014C040E050E068E070E0CE010E94280BFE
:101290008091E8008E778093E80088E0FE01A9E65F
:1012A000B1E001900D928A95E1F7DF91CF91089519
:1012B0008091E601811109C00E94C80C0E94250D91
:1012C0008091E20084608093E20008951092E6012C
:1012D0000895089508950C94201C809172018F5FE9
:1012E0008093720162E30E948924911135C01092AB
:1012F000720180917301882379F18091E701843034
:1013000049F58091E9008F709091EC0090FF02C048
:1013100090E801C090E0982B84E08093E9008091F0
:10132000EB0080FF14C08091EE0087FD03C00FC06A
:101330001092F1008091E80085FDFACF8091E800DD
:1013400080FF05C08091E8008E778093E8009F7051
:101350009093E90010927301089542E061EC81E0FE
:101360000E943E0C42E061EC82E00E943E0C42E0B2
:1013700061EC83E00E943E0C42E261EC84E00C945C
:101380003E0C8091E901833009F454C030F481307F
:1013900071F0823009F0A5C08CC08A3009F479C0A0
:1013A0008B3009F45FC0893009F09BC020C0809168
:1013B000E801813A09F095C08091E800877F809329
:1013C000E8008091EC019091ED01892B21F060E023
:1013D00080E090E003C068E089E691E070E00E9460
:1013E000770B8091E8008B778093E80008958091D7
:1013F000E801813209F075C08091EC019091ED0116
:10140000892B09F06EC08091E800877F8093E80007
:1014100005C08091E701882309F463C08091E8004A
:1014200082FFF7CF8091F100809371018091E800F5
:101430008B7753C08091E801813A09F052C08091C6
:10144000EC019091ED01892B09F04BC08091E800EF
:10145000877F8093E8008091E80080FFFCCF809137
:101460000B0136C08091E8018132D9F58091EC0101
:101470009091ED01892BA9F58091E800877F8093F9
:10148000E8000E94750C8091EA0180930B010C9496
:1014900015168091E801813221F58091E800877F5F
:1014A0008093E8000E94750C8091EB0180936801A5
:1014B00008958091E801813AA1F48091E800877F46
:1014C0008093E8008091E80080FFFCCF8091680164
:1014D0008093F1008091E8008E778093E8000C946F
:1014E000750C089584B7877F84BF88E10FB6F894A0
:1014F00080936000109260000FBE90E080E80FB60D
:10150000F89480936100909361000FBE0E943310A5
:101510000E94C80C0E94250D8091E2008460809397
:10152000E20078940E94C20F0E94351081E091E0A1
:101530000E94DF0F0BC00E94DD1B8091E501882314
:1015400029F00E94081C81110E94120B8091E70172
:10155000853089F30E943F10F9CF292F332723309C
:101560003105B1F04CF42130310509F44DC0223081
:10157000310509F04EC007C02132310541F1223258
:10158000310591F146C0E4E7F0E082E693E045C022
:1015900099278130910569F08230910589F0892B76
:1015A00009F037C0EEE5F3E0E491F0E08EE593E07A
:1015B00034C0E0E3F3E0E491F0E080E393E02DC099
:1015C000E4E0F3E0E491F0E084E093E026C06430EE
:1015D00000F5E62FF0E0EE0FFF1FEA5CFE4F808182
:1015E0009181E9E0F0E019C0643098F4E62FF0E072
:1015F000DF01AA0FBB1FA25CBE4F8D919C91EA5BDD
:10160000FE4FE081F0E009C0E2E1F0E086ED93E01A
:1016100004C0E0E0F0E080E090E0DA018D939C937C
:10162000CF01089580E189BD82E189BD09B400FE42
:10163000FDCF8091D8008F7D8093D8008091E0000D
:1016400082608093E0008091E00081FDFCCF0895EE
:10165000BF92CF92DF92EF92FF920F931F93CF939F
:10166000DF937C018B01EA010E94960CB82E811158
:1016700033C0209731F028813981021B130BE20E11
:10168000F31EC12CD12C23C08091E80085FD15C02C
:101690008091E8008E778093E800209749F0888158
:1016A00099818C0D9D1D9983888325E0B22E14C0ED
:1016B0000E94960C882359F00EC0F70181917F019A
:1016C0008093F10001501109FFEFCF1ADF0A0115D5
:1016D0001105D1F601C0B82E8B2DDF91CF911F914E
:1016E0000F91FF90EF90DF90CF90BF9008954091C1
:1016F000EE015091EF014617570748F0611571054B
:1017000039F44091E8004E774093E80001C0BA01F7
:10171000FC0140E033C08091E701882309F444C014
:10172000853009F443C08091E80083FD41C0809179
:10173000E80082FD33C08091E80080FF1FC09091D7
:10174000F3008091F200392F20E0A901482BCA0153
:1017500006C041914093F1006150710901966115F5
:10176000710519F088309105A0F341E0089709F060
:1017700040E08091E8008E778093E8006115710564
:1017800051F64111C8CF0AC08091E701882361F06A
:10179000853061F08091E80083FD0AC08091E80007
:1017A00082FFF2CF80E0089582E0089583E00895FB
:1017B00081E008954091EE015091EF0146175707DF
:1017C00048F06115710539F44091E8004E77409377
:1017D000E80001C0BA01FC0140E034C08091E7019B
:1017E000882309F445C0853009F444C08091E8009D
:1017F00083FD42C08091E80082FD34C08091E80002
:1018000080FF20C09091F3008091F200392F20E0FA
:10181000A901482BCA0107C044914093F1003196B9
:101820006150710901966115710519F088309105B3
:1018300098F341E0089709F040E08091E8008E7746
:101840008093E8006115710549F64111C7CF0AC0C0
:101850008091E701882361F0853061F08091E80094
:1018600083FD0AC08091E80082FFF2CF80E00895F6
:1018700082E0089583E0089581E00895982F2CC0B8
:101880009093E900981739F07091EC002091ED00E9
:101890005091F00003C0242F762F50E021FD02C0AC
:1018A0009F5F1AC03091EB003E7F3093EB00309188
:1018B000ED003D7F3093ED003091EB0031603093CF
:1018C000EB007093EC002093ED005093F00020911A
:1018D000EE0027FDE5CF07C0973090F28F70809320
:1018E000E90081E0089580E008958091E80187FD96
:1018F00005C08091E80080FF0EC012C08091E80012
:1019000082FD05C08091E7018111F8CF0895809193
:10191000E8008B7708C08091E7018111EACF089534
:101920008091E8008E778093E80008958091E4002C
:101930009091E50045E62091EC0020FD1FC023C0FA
:101940002091E701222391F0253091F02091EB00C6
:1019500025FD10C02091E4003091E50028173907DB
:1019600051F34150C90139F784E0089582E00895A8
:1019700083E0089581E0089580E008952091E800D3
:1019800020FFDECFF9CF2091E80022FFD9CFF4CF9E
:101990000E94360D0E943E0DE0EEF0E080818160F5
:1019A0008083E8EDF0E080818F77808319BCA7ED1C
:1019B000B0E08C918E7F8C9380818F7E808310929B
:1019C000E60108950F931F93CF93DF930E94360D86
:1019D0000E943E0DC8EDD0E088818F778883888192
:1019E0008068888388818F7D888319BC1092E70185
:1019F0001092E3011092E5011092E40100EE10E074
:101A0000F80180818B7F808388818160888342E0B8
:101A100060E080E00E943E0CE1EEF0E080818E7F8D
:101A20008083E2EEF0E08081816080838081886045
:101A30008083F80180818E7F8083888180618883A4
:101A4000DF91CF911F910F910895E8EDF0E0808133
:101A50008F7E8083E7EDF0E080818160808384E089
:101A600082BF81E08093E6010C94E20CE8EDF0E0A7
:101A700080818E7F80831092E20008951092DA00B8
:101A80001092E10008951F920F920FB60F92112449
:101A90002F933F934F935F936F937F938F939F9376
:101AA000AF93BF93EF93FF938091E10082FF0BC050
:101AB0008091E20082FF07C08091E1008B7F8093DC
:101AC000E1000E946D098091DA0080FF1FC08091C3
:101AD000D80080FF1BC08091DA008E7F8093DA00EF
:101AE0008091D90080FF0DC080E189BD82E189BD70
:101AF00009B400FEFDCF81E08093E7010E94580900
:101B000005C019BC1092E7010E9466098091E100AE
:101B100080FF19C08091E20080FF15C08091E20033
:101B20008E7F8093E2008091E20080618093E200EA
:101B30008091D80080628093D80019BC85E08093A2
:101B4000E7010E946A098091E10084FF30C0809122
:101B5000E20084FF2CC080E189BD82E189BD09B427
:101B600000FEFDCF8091D8008F7D8093D8008091BA
:101B7000E1008F7E8093E1008091E2008F7E809370
:101B8000E2008091E20081608093E2008091E301B5
:101B9000882311F084E007C08091E30087FF02C032
:101BA00083E001C081E08093E7010E946B0980918E
:101BB000E10083FF29C08091E20083FF25C080916E
:101BC000E100877F8093E10082E08093E70110923B
:101BD000E3018091E1008E7F8093E1008091E2003B
:101BE0008E7F8093E2008091E20080618093E2002A
:101BF00042E060E080E00E943E0C8091F00088604E
:101C00008093F0000E946909FF91EF91BF91AF911D
:101C10009F918F917F916F915F914F913F912F9104
:101C20000F900FBE0F901F9018951F920F920FB636
:101C30000F9211242F933F934F935F936F937F9352
:101C40008F939F93AF93BF93CF93EF93FF93809125
:101C5000E9008F709091EC0090FF02C090E801C005
:101C600090E0C92FC82B1092E9008091F000877F87
:101C70008093F00078940E94590E1092E9008091B0
:101C8000F00088608093F000CF70C093E900FF916E
:101C9000EF91CF91BF91AF919F918F917F916F9174
:101CA0005F914F913F912F910F900FBE0F901F901A
:101CB00018951F93CF93DF93CDB7DEB7AC970FB6D0
:101CC000F894DEBF0FBECDBFE8EEF1E08091F100E9
:101CD000819321E0E03FF207C9F70E94C10980919A
:101CE000E80083FF37C18091E8019091E9019530C8
:101CF00009F488C038F49130B1F170F0933009F0F4
:101D000029C131C0983009F4F8C0993009F404C1F0
:101D1000963009F01FC19DC0803821F0823809F04B
:101D200019C108C08091E4019091E501992389F0DF
:101D300082600FC08091EC019091ED018F70992726
:101D40008093E9008091EB0085FB882780F9109251
:101D5000E9009091E800977F9093E8008093F1006C
:101D60001092F100D5C0882319F0823009F0F2C03A
:101D70008F7121F0823009F0EDC00BC08091EA0133
:101D8000813009F0E7C0933009F080E08093E501ED
:101D90002FC08091EA0181112BC08091EC019091BC
:101DA000ED018F709927009709F4D4C08093E90062
:101DB0002091EB0020FF1CC02091E901233021F489
:101DC0008091EB00806212C09091EB009061909343
